:020000020000FC
:020000000BC033
:02000A00C9C467
:04000E00CBC3EBC3B2
:100016006CC000E60AB90FE90BB900E007B90EE3B8
:1000260008B900E004B90FEF05B90BEF0DBF04E006
:100036000EBFF1E0E0E0D1E0C0E0FF2499270FEF2A
:10004600A02E0FEDB02E0FEBC02E0FE9402E02E0D2
:10005600302E0AEFD02E0EEF902E01E0602E01E03A
:10006600202E44272227332751E06627772707E0EB
:100076000093FC0400E004BD01E005BD0BEF07BDE5
:100086000BEF08BD00E00093800008E000938100BC
:1000960000E00093890000E10093880000E00093EF
:1000A6006F0002E00093B00002E00093B1000FE998
:1000B6000093B3000AE00093B40006E000937000DA
:1000C60000EE00937C0005EA00937A0005E00093B9
:1000D6007B0001E003BF00E800BF04E00093680076
:1000E600789490936F008895FCCF6A94E1F4652E1E
:1000F600613091F4C030D20511F5182F150D179502
:1001060000917900011710F471E00EC0713061F4AE
:100116008FEF55247727772400917900099314E00F
:10012600CF3BD10730F5189500917900081708F4F0
:10013600802F501608F4502E739451F318950091A1
:100146007900081740F0501668F0099314E0CF3B89
:10015600D10778F41895802F099314E0CF3BD10787
:1001660040F41895502E099314E0CF3BD10708F4BC
:100176001895D1E0C0E008E0009381001895E0E012
:10018600F1E00EE1049FE00DF11D890103521040DC
:100196001FEF101B03E81F3F09F403E2153D09F4A6
:1001A60003E21A3A09F403E2103809F403E21F37AE
:1001B60009F403E2153509F403E21B3209F403E2FC
:1001C600103009F403E2033209F4BBB804BD01910F
:1001D60096BC0113D6BC01910113D6BC0191011343
:1001E600D6BC01910113D6BC01910113D6BC019175
:1001F6000113D6BC01910113D6BC01910113D6BCE3
:1002060001910113D6BC01910113D6BC01910113D2
:10021600D6BC01910113D6BC01910113D6BC019144
:100226000113D6BC01910113D6BC01910113D6BCB2
:1002360001910113D6BC01910113D6BC01910113A2
:10024600D6BC01910113D6BC01910113D6BC019114
:100256000113D6BC01910113D6BC01910113D6BC82
:1002660001910113D6BC01910113D6BC0191011372
:10027600D6BC01910113D6BC01910113D6BC0191E4
:1002860096BC0113D6BC01910113D6BC0191011392
:10029600D6BC01910113D6BC01910113D6BC0191C4
:1002A6000113D6BC01910113D6BC01910113D6BC32
:1002B60001910113D6BC01910113D6BC0191011322
:1002C600D6BC01910113D6BC01910113D6BC019194
:1002D6000113D6BC01910113D6BC01910113D6BC02
:1002E60001910113D6BC01910113D6BC01910113F2
:1002F600D6BC01910113D6BC01910113D6BC019164
:100306000113D6BC01910113D6BC01910113D6BCD1
:1003160001910113D6BC01910113D6BC01910113C1
:10032600D6BC01910113D6BC01910113D6BC019133
:100336000113D6BC019196BC0113D6BC01910113E1
:10034600D6BC01910113D6BC01910113D6BC019113
:100356000113D6BC01910113D6BC01910113D6BC81
:1003660001910113D6BC01910113D6BC0191011371
:10037600D6BC01910113D6BC01910113D6BC0191E3
:100386000113D6BC01910113D6BC01910113D6BC51
:1003960001910113D6BC01910113D6BC0191011341
:1003A600D6BC01910113D6BC01910113D6BC0191B3
:1003B6000113D6BC01910113D6BC01910113D6BC21
:1003C60001910113D6BC01910113D6BC0191011311
:1003D600D6BC01910113D6BC01910113D6BC019183
:1003E6000113D6BC01910113D6BC019196BC011331
:1003F600D6BC01910113D6BC01910113D6BC019163
:100406000113D6BC01910113D6BC01910113D6BCD0
:1004160001910113D6BC01910113D6BC01910113C0
:10042600D6BC01910113D6BC01910113D6BC019132
:100436000113D6BC01910113D6BC01910113D6BCA0
:1004460001910113D6BC01910113D6BC0191011390
:10045600D6BC01910113D6BC01910113D6BC019102
:100466000113D6BC01910113D6BC01910113D6BC70
:1004760001910113D6BC01910113D6BC0191011360
:10048600D6BC01910113D6BC01910113D6BC0191D2
:100496000113D6BC01910113D6BC01910113D6BC40
:1004A600019196BC0113D6BC01910113D6BC0191F2
:1004B6000113D6BC01910113D6BC01910113D6BC20
:1004C60001910113D6BC01910113D6BC0191011310
:1004D600D6BC01910113D6BC01910113D6BC019182
:1004E6000113D6BC01910113D6BC01910113D6BCF0
:1004F60001910113D6BC01910113D6BC01910113E0
:10050600D6BC01910113D6BC01910113D6BC019151
:100516000113D6BC01910113D6BC01910113D6BCBF
:1005260001910113D6BC01910113D6BC01910113AF
:10053600D6BC01910113D6BC01910113D6BC019121
:100546000113D6BC01910113D6BC01910113D6BC8F
:1005560001910113D6BC019196BC0113D6BC019141
:100566000113D6BC01910113D6BC01910113D6BC6F
:1005760001910113D6BC01910113D6BC019101135F
:10058600D6BC01910113D6BC01910113D6BC0191D1
:100596000113D6BC01910113D6BC01910113D6BC3F
:1005A60001910113D6BC01910113D6BC019101132F
:1005B600D6BC01910113D6BC01910113D6BC0191A1
:1005C6000113D6BC01910113D6BC01910113D6BC0F
:1005D60001910113D6BC01910113D6BC01910113FF
:1005E600D6BC01910113D6BC01910113D6BC019171
:1005F6000113D6BC01910113D6BC01910113D6BCDF
:1006060001910113D6BC01910113D6BC019196BC90
:100616000113D6BC01910113D6BC01910113D6BCBE
:1006260001910113D6BC01910113D6BC01910113AE
:10063600D6BC01910113D6BC01910113D6BC019120
:100646000113D6BC01910113D6BC01910113D6BC8E
:1006560001910113D6BC01910113D6BC019101137E
:10066600D6BC01910113D6BC01910113D6BC0191F0
:100676000113D6BC01910113D6BC01910113D6BC5E
:1006860001910113D6BC01910113D6BC019101134E
:10069600D6BC01910113D6BC01910113D6BC0191C0
:1006A6000113D6BC01910113D6BC01910113D6BC2E
:1006B60001910113D6BC01910113D6BC019101131E
:1006C600D6BC019196BC0113D6BC01910113D6BCD0
:1006D60001910113D6BC01910113D6BC01910113FE
:1006E600D6BC01910113D6BC01910113D6BC019170
:1006F6000113D6BC01910113D6BC01910113D6BCDE
:1007060001910113D6BC01910113D6BC01910113CD
:10071600D6BC01910113D6BC01910113D6BC01913F
:100726000113D6BC01910113D6BC01910113D6BCAD
:1007360001910113D6BC01910113D6BC019101139D
:10074600D6BC01910113D6BC01910113D6BC01910F
:100756000113D6BC01910113D6BC01910113D6BC7D
:1007660001910113D6BC01910113D6BC019101136D
:10077600D6BC01910113D6BC01910113D6BC000071
:10078600000096BC0000D6BC00E004BDCBB80895BE
:100796002227332783940AC006E90093B4000CC0CD
:1007A6004BB8220D3F1D2833320590F727303F0501
:1007B60098F30AE00093B40021303F0579F433D072
:1007C600C030D20559F4613049F4082D1091FC046B
:1007D600153008F007700F7109F4E3D030926F00FE
:1007E6001895CBB81FEF00918100083009F4112746
:1007F6000091FC04053008F011271F1113C02332A5
:100806003F0548F02332320530F400000EE10A9528
:10081600F1F7B5DC07C02432320520F02B32320561
:1008260008F44FD218950091FE04003019F00A958D
:100836000093FE041091FF0406B10E730093FF04AB
:100846001017C1F01091FE041030A1F401FF09C089
:1008560002FF09C003FF09C004FF09C005FF09C064
:1008660009C042D007C045D005C048D003C050D00B
:1008760001C058D015E001FF1093FE0402FF10934B
:10088600FE0403FF1093FE0404FF1093FE0405FF0D
:100896001093FE040E3329F01091FD041395109366
:1008A600FD041091FE04103019F410E01093FD04BD
:1008B6001091FD041233B9F41EE21093FD0401FFFA
:1008C60009C002FF09C003FF09C004FF09C005FFF4
:1008D60009C009C02BD007C02BD005C02BD003C040
:1008E6002BD001C02BD0089500E0401709F04A959F
:1008F600089508E1401708F4439508950091FC0413
:10090600013028F00A950093FC041AD04AD00895C5
:100916000091FC04093128F403950093FC0410D0DF
:1009260040D0089560E00CD03CD00895DDCF089506
:10093600E0CF0895E3CF0895EBCF089561E00895E1
:10094600D1E0C0E00FEF0993099309930993099346
:1009560009930993099309930993099309930993B1
:1009660009930993099309930993099309930993A1
:100976000993099309930993099309930993099391
:10098600099314E0CF3BD107F0F2D1E0C0E008951F
:1009960004E000936D00089500E000936D0009D017
:1009A6001895613031F008E00093810009B102FF2B
:1009B600EFCF992751E0D1E0C0E00091FC04E7EECB
:1009C600F4E0E00FFF1D099419C026C033C040C0F3
:1009D6004DC05AC066C072C07EC08AC096C0A2C052
:1009E600AEC0BAC0C6C0D2C0DEC0EAC0F6C002C140
:1009F6000EC11BC128C135C142C14FC102EA0093D5
:100A06007A0009E00093810000E00093890000E28B
:100A160000938800932D4FC103EA00937A0009E002
:100A26000093810000E00093890001E400938800B0
:100A3600932D41C103EA00937A0009E000938100F7
:100A460000E00093890004E800938800932D33C1E9
:100A560004EA00937A0009E00093810001E0009324
:100A660089000CE400938800932D25C104EA0093C5
:100A76007A0009E00093810002E0009389000AE908
:100A860000938800932D17C105EA00937A0009E0C8
:100A96000093810005E00093890004E30093880039
:100AA6000AC106EA00937A0009E0009381000DE08E
:100AB6000093890004E000938800FDC006EA0093D5
:100AC6007A0009E0009381000AE1009389000AE0B8
:100AD60000938800F0C007EA00937A0009E00093CB
:100AE600810004E30093890004E100938800E3C0D9
:100AF60007EA00937A0009E00093810002E8009378
:100B0600890004E300938800D6C007EA00937A00C0
:100B16000AE00093810000E2009389000CE800934C
:100B26008800C9C007EA00937A000AE000938100B2
:100B360001E4009389000AE100938800BCC007EA3B
:100B460000937A000AE00093810002EA009389008C
:100B560001EC00938800AFC007EA00937A000BE02F
:100B66000093810008E20093890000EB009388005F
:100B7600A2C007EA00937A000BE00093810001E52A
:100B86000093890000E60093880095C007EA009369
:100B96007A000BE0009381000BEC0093890002E7DA
:100BA6000093880088C007EA00937A000CE000935F
:100BB600810005E60093890009EB009388007BC05D
:100BC60007EA00937A000CE0009381000BEC009397
:100BD600890002E7009388006EC007EA00937A0056
:100BE6000DE0009381000FE70093890007E2009370
:100BF600880061C007EA00937A000DE00093810047
:100C06000EEF009389000FE40093880054C007EAB2
:100C160000937A000DE0009381000EEF00938900A7
:100C26000FE40093880053E046C007EA00937A0079
:100C36000DE0009381000EEF009389000FE400930E
:100C4600880056E038C007EA00937A000DE000936A
:100C560081000EEF009389000FE40093880052E1B3
:100C66002AC007EA00937A000DE0009381000EEF98
:100C7600009389000FE40093880054E21CC007EA41
:100C860000937A000DE0009381000EEF0093890037
:100C96000FE4009388005CE60EC007EA00937A0032
:100CA6000DE0009381000EEF009389000FE400939E
:100CB600880058ED00C0F0928500F0928400652E01
:100CC6000895E22E04E2E01A0BE40A95F1F785D1C5
:100CD6000091FC04E2E7F6E0E00FFF1D099419C05D
:100CE6001DC022C027C02CC02FC032C035C039C09D
:100CF6003DC041C046C04BC050C052C054C056C093
:100D060059C05CC05FC063C067C06CC071C073C0AF
:100D160075C0E3D1D6D1E7D1ECD173C0D5D1D1D14D
:100D2600D0D1E1D1E6D16DC0D2D1CBD1CAD1DBD100
:100D3600E0D167C0D2D1C5D1C4D1D5D1DAD161C095
:100D4600C3D1D4D1D6D15DC0C2D1D0D1D2D159C0B0
:100D5600C4D1CCD1CED155C0B7D1B3D1C7D1C9D169
:100D660050C0B5D1AED1C2D1C4D14BC0B6D1A9D134
:100D7600BDD1BFD146C0A8D1A4D1A3D1B7D1B9D1D5
:100D860040C0A5D19ED19DD1B1D1B3D13AC0A5D194
:100D960098D197D1ABD1ADD134C096D1AAD131C0BB
:100DA60096D1A7D12EC099D1A4D12BC08DD189D1EE
:100DB600A0D127C08CD185D19CD123C08ED181D121
:100DC60098D11FC081D17DD17CD193D11AC085D154
:100DD6008DD198D19DD115C077D173D187D192D1BC
:100DE60097D10FC077D16DD181D18CD191D109C066
:100DF6006BD182D106C06ED17FD103C071D17CD1B7
:100E060000C089D17CD17ED180D1613011F489D1E5
:100E16000CC000918100083011F080D106C000910D
:100E26006D00043011F480D100C008958E01115078
:100E36001695079516950795169507951695079590
:100E460016950795C030D20509F40FEF0F3F21F430
:100E56000000000000000000003021F4ABB80000E4
:100E66000000CBB8013021F4ABB800000000CBB8CD
:100E7600023021F4ABB800000000CBB8033021F4F7
:100E8600ABB800000000CBB8043021F4ABB80000CA
:100E96000000CBB80000053021F4ABB8000000001C
:100EA600CBB8063021F4ABB800000000CBB8073051
:100EB60021F4ABB800000000CBB8083021F4ABB881
:100EC60000000000CBB8093021F4ABB800000000E8
:100ED600CBB800000A3021F4ABB800000000CBB854
:100EE6000B3021F4ABB800000000CBB80C3021F475
:100EF600ABB800000000CBB80D3021F4ABB8000051
:100F06000000CBB80E3021F4ABB800000000CBB81F
:100F160000000F3021F4ABB800000000CBB8003160
:100F260021F4ABB800000000CBB8013121F4ABB816
:100F360000000000CBB8023121F4ABB8000000007D
:100F4600CBB8033121F4ABB800000000CBB80000E9
:100F5600043121F4ABB800000000CBB8053121F410
:100F6600ABB800000000CBB8063121F4ABB80000E6
:100F76000000CBB8073121F4ABB800000000CBB8B5
:100F8600083121F4ABB800000000CBB800000931ED
:100F960021F4ABB800000000CBB80A3121F4ABB89D
:100FA60000000000CBB80B3121F4ABB80000000004
:100FB600CBB80C3121F4ABB800000000CBB80D3132
:100FC60021F4ABB800000000CBB800000000000020
:100FD60070C000000000000029CF05E00E15C9F31F
:100FE60006E00E15C9F303E00A95F1F700000000CC
:100FF60000E00E1521F004E00E1521F00DC00000F2
:1010060000000000000000000000BBB80000000067
:1010160001E20A95F1F74DC011274030BBB809F43B
:101026004AD0413009F447D0423009F444D0433025
:1010360009F441D0443009F43ED0453009F43BD0A0
:10104600463009F438D0473009F435D0483009F431
:1010560032D0493009F42FD04A3009F42CD04B3025
:1010660009F429D04C3009F426D04D3009F423D0A8
:101076004E3009F420D04F3009F41DD0403109F428
:101086001AD0413109F417D0423109F414D0433152
:1010960009F411D0443109F40ED0453109F40BD0CE
:1010A600463109F408D0473109F405D0483109F42E
:1010B60002D0CBB80895CBB807E00A95F1F7BBB8D4
:1010C6000895F1E1ECE733C0F1E1E4E830C0F1E185
:1010D600ECE82DC0F1E1E4E92AC0F1E1ECE927C032
:1010E600F1E1E4EA24C0F1E1ECEA21C0F1E1E4EB4C
:1010F6001EC0F1E1ECEB1BC0F1E1E4EC18C0F1E13C
:10110600ECEC15C0F1E1E4ED12C0F1E1ECED0FC03D
:10111600F1E1E4EE0CC0F1E1ECEE09C0F1E1E4EF3F
:1011260006C0F1E1ECEF03C0F2E1E4E000C0EE0D31
:10113600FF1D049104FFCBB804FDABB8000000000E
:1011460003FFCBB803FDABB80000000002FFCBB82D
:1011560002FDABB80000000001FFCBB801FDABB843
:101166000000000000FFCBB800FDABB80000000097
:101176000000CBB808950C12121212120C000206CF
:101186000A02020202000C12020404081E000C12DB
:10119600020402120C001E101C0202120C000C1299
:1011A600101C12120C000000121212120E00000087
:1011B6001E151515150000000E100C021C0010104F
:1011C6001C121212120002020E1212120E0004005B
:1011D6000C0404040E00000011110A0A04000000A9
:1011E6001C12121212000202040404080800000471
:1011F600021F0204000010181C1E1C1810001F11EC
:06120600171317111F0071
:00000001FF
